S10D00B100002023000600000000F8
S12302007E03557E03837EE1AC7EE1D17EE1AC7EE1D11FFF415050454E440012DD41001272
S1230220DD424F54544F4D00098E4200098E4348414E4745000DCB434F5059000FF3434F4B
S1230240000FF343000DCB44454C455445000C8A44000C8A455850414E4400125C4558503F
S123026000125C46494E440009CF460009CF47415000141348454144455200111B480011C8
S12302801B494E53455254000AC849000AC84C4F470009894D4F5645000FD44D4F000FD470
S12302A04E4558540009CC4E554D4245525300091D4E5500091D4E0009CC4F5645524C412F
S12302C059000F214F000F215052494E54000877500008775245414400142A52454E554D56
S12302E04245520006A552454E0006A55245504C414345000C8752000C8753415645001330
S12303009D5345540011CC53544F50000989530009895441420010D0544F5000099D540012
S1230320099D5645524946590009635600096357524954450013AD570013AD580009785A7B
S12303404F4E4500117E5A00117E004E45572046494C453A048E01FFCE1600DF97DF99CEA9
S12303600203FFA048CE0001DF5ECE0136DF60864697964F979D4A978F976A976BCE034B32
S1230380BD0483DE97DF487F006C8E01FFDF40DE48DF4ACE006D4FA700088C008E26F8DE43
S12303A040968F27067F008F7E0AEA966C2622978ECE00BBBD044E8623BD0209BD0499272E
S12303C0C9A700810D2705BD04BB20F0CE00BBDF447F006CBD04D24F9775978CDF4ADE4470
S12303E0BD0492DF44813D260808DF44CE0AA52044BD06632605CE0877203ADF40CE021490
S1230400DF9B6D002723A100260CDE4408A600DF44DE9B0820EA086D0026FB0808086D003B
S1230420271F09DF9BDE4020E408EE008C0AC82604967F260ABD082126254F977297736E09
S123044000CE044C8D3D7F006C7E038A3F04DF42CE04588D30DE42390D0A0000000004CE2D
S1230460046420E04E4F2053554348204C494E4504CE047620CE53594E54415820455252AE
S12304804F52048DC9A6008104270DBD02090820F408A600812027F939BD02068108260BF3
S12304A08C00BB2715097A008E20EE8118270B811F2204810D26E27C008E39088C0143262E
S12304C0F98607BD0209BD0206810826F4097A008E398DBE813D270A7C0075BD073BC1012C
S12304E02303DE4A39272320148D03DF93397F008CBD0738C10123037E0471277D7F008C27
S123050091B4262E08BD0492DF44BD0755DF40DE4A9690A100260A9691A10126049692A1AD
S12305200224037A008CDE40BD07AB27B7D7747E07F0BD0663260A7D007627A6DE4A7E0899
S12305400F8121260808DF44DE997E07F0815E26097A008C08DF44DE9739812B2707812D2C
S123056026477A008C08BD0738C101270D233AD6752785BD07A3DE4A201ABD0755DE4A7D2F
S123058000752608BD0838271FBD082ABD08382717BD082ABD06C3BD082127F0967326089E
S12305A0BD083826037C007F398D4F8D6DDE4ABD06C3080808BD065ABD082A2722C60DE138
S12305C00027030820F2968526DE089C99270609968526D409BD06C3BD0821261720D3BDCA
S12305E0065ABD06CD7D007027E65F96852605BD07F6DF9339860197733997955F08DF4E79
S1230600A6008D5F270891952704085C20F2DF50D77B8D4F270108DF4439BD073B7F006D7A
S1230620C1012617BD07558D1B25108D22220C7C006D969097629691976339965E976296FF
S12306405F976339D690D15E2604D691D15F39D690D1602604D691D16139966297909663CA
S1230660979139810D270291B5398601D67C270C2A0286109B9219979225013986015F9BC2
S123068091199791179990199790399690A7009691A7019692A70239A6009790A601979189
S12306A0A602979239BD09A4DE977F007CBD07A38DB88DD7BD080F967327F59683270139CF
S12306C07E08A2968C2B037E080F7E07F07F0070D67B26067C0070DF5C39C60DDF4CDF5C8F
S12306E0DE4EDF56A600DE4CE100271DA100271D7D006D26147D0070262208DF5C3637BDF5
S1230700067CBD064F333223DF7F00703908DF4C7C0070DE56089C50270F20C6DE5C08BD50
S1230720067CBD064F23A620E0D67B270837BD067C335A26F6DE5C39BD0492DF44A6005FCB
S1230740812F2310813922025C3981402306815A2202C602398D4C8DE2C1012707812E2747
S123076017DF443908840FC6047800917900905A26F79B91979120DFC602D789088DBCC187
S12307800127044F092002840FC6047800925A26FA9B9297927A008926E2088D9EC1012751
S12307A0F920BE4F97909791979239D6909691DE979C9926057C00735C39E100221C26F83B
S12307C0A101221626F2D692E102220E26EA7D008426057D008326E05F397D008326F98D22
S12307E005D6900820CB36860D08A10026FB32399C972717C601099C97270DA600810D2697
S1230800F55A2AF208C601395D27FC7C0072399C992606C601D77320D78DCB089C9927F3A2
S1230820397D007226037D0073398699169B9119979117999019979096902602969139DF8B
S12308404ABD07E6DF5A4F978D09090909E600C10D2709E603C12026034C20F0978E080868
S12308600808DF58BD0D43DE4A966B27058D40BD07F0DF48DF4A398D2FDE44BD04E9DE4A11
S12308807C008ADF489C9326037F008A8D21968A270B968C27EF0909BD07F020E8BD07F00C
S12308A0DF48BD09B57E038ADE979C9927F439BD044E966A26068D15080820038D160908C5
S12308C0A600810D2705BD020920F408398620BD02090C39966A272E8DF3C6020CA6008510
S12308E0F025022706BD09130D20028DE0A600C5FE2706850F250227058D1C0D20028DCD8C
S1230900085A27072AD7863D7E0209862EBD02090D20CA44444444840F8B3020EB8D18274E
S1230920072B0A7F006A200843976A200373006ADE4ADF487E08A2DE44BD0492DF44DF40F4
S1230940CE09467E04004F4E0009564F46460009580D00095B004F39860139DE4409DF44B5
S123096086FF398DD227072B0A7F006B200843976B200373006B20B88D2ACE0982BD04856D
S123098020AE000000000000048D197EE0E38D14BD08A8DE99BD07F0DF487E08A28D05BDC3
S12309A008A820F4DE44BD0492810D270491B52601397E0471DE44860DD6B5A100270CE1B3
S12309C00027030820F508DF44976C397C0076BD08A87C00758D71DE93BD0821272AD67623
S12309E02643200496772640CE0A31BD0483DE5E8C00012607DE608C01362706CE0A3BBDB2
S1230A0004857F006C7E038ADE939C4A271ADF4AD6782711D6762603BD083FBD0A83BD0884
S1230A202127E52006BD083F7E08A2D67626F620B34E4F5420464F554E44042E2E2E5A4F34
S1230A404E4553204F4B3F04DE44DF467F00777F0078BD04E9DE44BD0738C1012709812A16
S1230A6026177C0077200FBD0755BD0838270ABD082A27058D047C0078399690976E9691A1
S1230A80976F399677260F966E9790966F9791BD082A270B8DE49685260ADE467E04E97F8E
S1230AA0007820F239BD08A8DE447F007D7C00847C007E96742620DE4ADF93BD06987C0029
S1230AC081968E97827E0CBBDE447F007DA600810D27177C008408DF44CE00BB968E9C44C7
S1230AE027044A0820F88B03978EDE4ADF48967E2706967227142025BD0698967F270B9C54
S1230B009927075FD790D7912013BD080FE6029673270A5FDE999C972603BD07A3DF58964D
S1230B207E262C967327057F0092201C967D26189692D7829A82270D967F27037F00928667
S1230B4001977C20037A007CBD066A96842704DE44202D7F007FBD044ECE0090BD08D47F00
S1230B60008D8603978E977DCE00BBBD049927E3810D2707A700BD04BB20F0A700CE00BB16
S1230B80DF44A60091B42640968E8003978E08DF40DE4ABD080F7D0073261A7C0083D69059
S1230BA09691BD07BA260E4F977C9792BD06B0CE0BF2BD0483DE407D00842706DE4ADF48B0
S1230BC020037C006C7E038A8D3EDE40DF4ABD068B080808DF40DE44A60008DF44DE40A7AC
S1230BE00008DF40810D26EEBD1285968426A07E0AEA534F4D45204C494E45532052454EAE
S1230C00554D4245524544047F0089DE58DF409C9926037C0089DE99DF58D68D968E2603AA
S1230C205D2737BC02122726087D008C2604DF42200C7D008B270EDF42DE4A08DF4ADE9328
S1230C4008DF93DE424D26015A4A26D720D2CE0C77BD04837F006C7E038ADF99DF5A968994
S1230C602614DF5ADE589C40270C09A600DF58DE5A09A70020EC394E4F5420454E4F554716
S1230C804820524F4F4D047C0081DE44BD04E9BD08212727CE0D7FBD0483CE00BBBD049929
S1230CA027F2A70008810D26F4CE00BBBD049281592708CE0DA3BD04832060DE4A968C2728
S1230CC015BD080F96732702DE99DF5ADE93DF48DF58DE5A2011DF58DF48DE93BD080F96D4
S1230CE0732702DE99DF5A4F5F9C5827074C26015C0920F5978ED78D8D499681271DDE4807
S1230D00BD07F0967E262C96722708BD07A3DF4A7E0B1DDF4A7F007D7E0AEADE489C992630
S1230D200DBD07F0DF40CE0DB4BD0483DE40DF487E08A2DF4A9682978E4F977D978DDE4480
S1230D407E0AD7DE5A9C5827359C99270EA60008DF5ADE58A70008DF5820E8D68D968E2686
S1230D60035D2718097D008C2609DF42DE9309DF93DE424D26015A4A26EA20E5DF99395430
S1230D804152474554204E4F542052454143484544210D0A00000000594F5520535552452B
S1230DA03F20044E4F204C494E45532044454C4554454404424F54544F4D204F4620464940
S1230DC04C45205245414348454404BD08A8DE44BD0738BD066327035D27037E0F047C00FF
S1230DE085BD05FA5FA600BD0663270891952704085C20F1DF66D786BD0663270108DF4473
S1230E00DE4A080808DF64BD0F077F0085BD0A487C0085BD0F147F006DDE6EDF68967827D0
S1230E2007967B26037E0F04DE4A9C9326037C0088BD063B7F0079DE64BD065ABD05B82069
S1230E40107F0079DE64BD065ABD064F227ABD05DF96909762969197635D266C5CD7879659
S1230E6078270E9677260ABD0A87DE5C08DF6420D07C0079DE68270486019778DF6EDE5C3E
S1230E80DF58D67B27107F008DD78E2704085A20FADF5ABD0D43D68627237F008DD78EDE3C
S1230EA05CDF58BD0C08D68EDE5008A600DF40DE5CA70008DF5CDF64DE405A26ED96772745
S1230EC01CDE5CDF647E0E447F0078DE68270486019778DF6E9687260496882627DE4A96EA
S1230EE0792703BD083F968827067F00797E08A2BD06C3DF4A9C9326037C0088080808DFDA
S1230F00647E0E317E0441DE4EDF52DE50DF54967B977139DE52DF4EDE54DF509671977B02
S1230F2039BD08A8862097957F008CDE44A600810D2712BD073B5D27037E0471979508A648
S1230F4000810D262CDE4ABD08AF966A2605CE0FD22003CE0FCABD0483CE00BBBD0499271F
S1230F60E4810D2707A700BD04BB20F0A700CE00BBDF44C60DDE4A080808DF40DE44A6004D
S1230F8008DF44810D273BDE407D008C2608E100270B91952702A70008DF4020DF968C2666
S1230FA0214F978DDE444CE10027030820F8978EDE40DF588601978CBD0C08C60DDE44090D
S1230FC020BCDE4ABD083F7E038A204F5645524C415920047C00808D1A968B978CDE93DF5D
S1230FE05ADE4ADF58DE48DF93BD0D43DE93DF487E08A2DE447C00767C0075BD04E99C99EB
S1231000271A7F00757F00769C9726049C4A2704968C978B7F008CBD082127037E045FBD37
S123102007E608DF58DE44BD04E9BD082126ED7D008C2608DE4ADF40DE932006DE93DF4016
S1231040DE4ABD07E608DF93DE40DF4A4F5F084C26015C9C9327109C5826F3CE10B4BD04AE
S1231060837F006C7E038A978ED78D8601978CBD0C08DE5ADF48DE58DF42DE93DF58DE4A69
S1231080DF40BD0C64DE427F0072BD07F096722718BD07A37C0083BD06B0DE48BD07F0DF62
S12310A04896802701397E08A2BD06984F9792BD080F20E0534F55524345204F5645524C25
S12310C04150532044455354494E4154494F4E04CE009DDF9BDE44BD0492DF44BD066327F8
S12310E02FBD073BC1012707222E08DF4420E6BD0755DF445FBD083827165C37BD082A33C3
S123110026F8DE9BE70008DF9B8C00B1270220C54FDE9BA7007E09307E0471CE009DDF9B82
S1231120DE44BD0492BD0663271CBD073BC10126E7BD0755DF44BD083827405F5C37BD08A8
S12311402A3326F8D796BD07A3BD044E966A2708C608BD08CD5A26FABD08CD5F37BD067CBD
S1231160335CDE9BE100260A862DBD020908DF9B20059691BD0917D19626E17E0930DE44E5
S1231180BD0492BD0663270ABD073BC101270A223808DF44CE00012007BD0755DF44DE908A
S12311A0DF5EDE44BD0492BD0663270CBD073BC101270A22140820ECCE01362007BD07559F
S12311C0DF44DE90DF607E09307E0441DE44BD0492DF44DF40CE12417E0400CE00B2200DBA
S12311E0CE00B32008CE00B52003CE00B4DF40DE44BD0492813D263F8D40263B8D3C260442
S12312004F36200FBD073B5D262D810D2729368D29262408DF44BD09A432DE408C00B32609
S1231220074D260E8620200A8C00B426054D26028623A7007E09307E047108BD0492812775
S1231240395441420011DB46494C4C0011E0454F4C0011E54C494E4F0011EA00BD08A8DE28
S123126044BD04E9DE4A8601978ADF489C9326037F008A8D10968A2709DE4ABD06C3DF4A60
S123128020E87E08A296B291B32751CE009DDF9BE60027485FD78DDE4A9C9926037E038A88
S12312A00808085CA600810D273291B227030820F2DF40DE9BE100241E86FF4C5CE10026B3
S12312C0FA978EDE40DF58BD0C08D68E5C96B3A700085A26FA20AE08A60026D939BD08A872
S12312E0DE44BD0492BD066326037E0471BD073B5D26F7BD05FABD073BC1012613BD0755EB
S1231300BD0838270B4F4C36BD082A3226F8977ABD0F07DE44BD04E9BD0F147F008D7C0072
S12313208ADE4A9C9326037F008A080808967A260609BD07E62037165A271CA600810D272A
S1231340030820F4DF58D78E37BD0C08338620A700085A26FA2017DF58DF40A600810D27DC
S123136004085C20F6D78EDF5ABD0D43DE40DF58967B2712978EBD0C08DE50DF58DE4EDF3B
S123138040BD0C64DE5A5FBD07F6BD083F968A2707BD06C3DF4A208BDF487E08A2BD09A426
S12313A0DE97DF58DE99DF5A8D297E0930BD08A8DE44BD04E9968C260CBD07E608DF5ADE0A
S12313C04ADF58200ADF58DE4ABD07E608DF5A8D0220D796B9BD020F8D2BDE589C5A271551
S12313E0080808A600810D2706BD020F0820F4BD020F0820E7861ABD020FCEFFFF0926FD43
S123140096BABD020F96B62709CEFFFF0926FD4A20F539BD09A496B9BD020F8DE8C6284F65
S1231420BD020F5A26F98DD820A7BD09A496B7BD020F8DD1BD07A3DE99DF409C972708BD36
S123144007F0BD0698DE998D358D338D31BD020C810D270C811A270C811F23F18D2120EDB6
S12314608D1D20E35FBD07F6DF997C008396B8BD020F9C402705DE40BD06B07E09904FBC54
S115148002122704A7000839BD020C811A26F920D30DAA
S105A048020010
S9030000FC
